:020000040000FA
:0400000037EF0CF0DA
:0400080010EF10F0F5
:0800180000EF20F010003DEFA5
:1000200000F088EF09F051EF0CF07BEF07F094EF50
:100030000BF050EF04F06EEF08F01FEF0CF07CEFC8
:1000400006F04BEF0CF002EF0AF072EF05F055EFFF
:100050000AF0F1EF0BF0CAEF0BF0AFEF0BF074EF1B
:100060000BF041EF0CF02BEF0CF011EF0CF0F9EF6F
:1000700002F012EF03F0EDEF02F000C0E5FF01C067
:10008000E5FF02C0E5FF03C0E5FF04C0E5FF69A48A
:1000900005D068A403D06D926994689469A003D0D8
:1000A00068B088EC09F069A805D068A803D0698415
:1000B00068986D8269AA42D068AA40D0006A70B080
:1000C000002A0050010A39E15E50030DF3CF00F021
:1000D000F4CF01F0000184510026855101228651A0
:1000E000026A022200C0E9FF01C0F3FF0250AFEC38
:1000F0000BF0006EF3CF01F0F4CF02F000C0E9FF87
:1001000001C0F3FF0250AFEC0BF0006EF3CF01F033
:10011000F4CF02F0F2CFE5FFF29E0500380EFD6E3F
:10012000010EFE6E000EFF6EE450F26E02C0FBFF89
:1001300001C0FAFF0050F96E7090689A030E5F5C80
:10014000D8A015D169A613D168A611D16CB4B9D0C5
:100150006C50E838E8440F0B006E0024040DF3CF18
:1001600000F0000E0026040E016A00BE01680122A4
:1001700000C0E9FF01C0EAFFEF50E840E8400F0B84
:100180000D0A01E04FD05E50030DF3CF00F0F4CF25
:1001900001F0000187510026885101228951026A2D
:1001A000022200C0E9FF01C0F3FF0250AFEC0BF0E8
:1001B000006EF3CF01F0F4CF02F06C50E838E84461
:1001C0000F0BE56AE56EE56A030EE56E55EC0AF085
:1001D000036EF3CF04F0040EE12603500026045012
:1001E0000122E86A022200C0E9FF01C0F3FF0250C9
:1001F000AFEC0BF0006EF3CF01F0F4CF02F0F2CFD2
:10020000E5FFF29E0500220EFD6E020EFE6E000E50
:10021000FF6EE450F26E02C0FBFF01C0FAFF005017
:10022000F96EA4D05E50030DF3CF00F0F4CF01F0CF
:1002300000018A5100268B5101228C51026A022250
:1002400000C0E9FF01C0F3FF0250AFEC0BF0006EFD
:10025000F3CF01F0F4CF02F06C50E838E8440F0B14
:10026000E56AE56EE56A030EE56E55EC0AF0036E8D
:10027000F3CF04F0040EE1260350002604500122BF
:10028000E86A022200C0E9FF01C0F3FF0250AFECB0
:100290000BF0006EF3CF01F0F4CF02F0F2CFE5FFE8
:1002A000F29E0500C00EFD6E020EFE6E000EFF6E89
:1002B000E450F26E02C0FBFF01C0FAFF0050F96E7D
:1002C00055D0006A6CB4002A0050010A01E04ED0FB
:1002D0005E50030DF3CF00F0F4CF01F000018D511B
:1002E00000268E5101228F51026A022200C0E9FFCE
:1002F00001C0F3FF0250AFEC0BF0006EF3CF01F042
:10030000F4CF02F06C50E838E8440F0BE56AE56E74
:10031000E56A030EE56E55EC0AF0036EF3CF04F0C8
:10032000040EE1260350002604500122E86A02224E
:1003300000C0E9FF01C0F3FF0250AFEC0BF0006E0C
:10034000F3CF01F0F4CF02F0F2CFE5FFF29E05000B
:100350006C0EFD6E030EFE6E000EFF6EE450F26E2C
:1003600002C0FBFF01C0FAFF0050F96E6896E4CFAF
:1003700004F0E4CF03F0E4CF02F0E4CF01F0E4CFE7
:1003800000F0120012010002FF00FF08D804AAFECC
:1003900001000102030209021200010104C0000968
:1003A00004000000FFFFFF0409022000010205C055
:1003B000000904000002FFFFFF05070501024000DD
:1003C0000007058202400000960300A80300040312
:1003D000090426034A00650061006E002D005000EC
:1003E0006900650072007200650020004D00410048
:1003F0004E0044004F004E002203500069006E0082
:100400006700750069006E006F00200050007200E8
:100410006F006A006500630074000403310010037C
:10042000440065006600610075006C0074000C03F8
:1004300046006C00610073006800CE0300D2030028
:10044000F803001A04001E04002E0400281700AC54
:100450001800AC1800AC1800AC1800AC1800AC18B0
:1004600000AC1800AC1800AC1800AC1800AC1800B8
:10047000AC1800AC1800AC1800AC18002817003EEF
:100480001800961800AC1800AC1800AC1800AC1896
:1004900000AC1800AC1800AC1800AC1800AC180088
:1004A000AC1800AC1800AC1800AC18004C04004CA0
:1004B00004007C040000A00800AC1800AC1800ACDC
:1004C0001800AC1800AC1800AC1800AC1800AC1840
:1004D00000AC1800AC1800AC1800AC1800AC180048
:1004E000AC1800AC1800A00800AC1800041400AC54
:1004F0001800AC1800AC1800AC1800AC1800AC1810
:1005000000AC1800AC1800AC1800AC1800AC180017
:10051000AC1800AC1800B60400B60400E6040000F5
:10052000281700AC1800AC1800AC1800AC1800ACD0
:100530001800AC1800AC1800AC1800AC1800AC18CF
:1005400000AC1800AC1800AC1800AC1800AC1800D7
:10055000281700F80C00AC1800AC1800AC1800AC60
:100560001800AC1800AC1800AC1800AC1800AC189F
:1005700000AC1800AC1800AC1800AC1800AC1800A7
:1005800020050020050050050000DC1000AC18001C
:10059000AC1800AC1800AC1800AC1800AC1800ACDB
:1005A0001800AC1800AC1800AC1800AC1800AC185F
:1005B00000AC1800AC1800AC18008A05008A0500D1
:1005C0008A0500000301000000FF1F000300200057
:1005D000FF7F00010000300D0030E8060000E85009
:1005E00007E000D000D000D000D00000E82EFAD7FD
:1005F0001200E806E56E090E12EC03F0630EEDEC56
:1006000002F0E4500EE000D0E56E090E12EC03F0AB
:10061000630EEDEC02F000D000D00000E450E82EB4
:10062000F3D71200E806E56E630EEDEC02F0E4503D
:100630000BE000D0E56E630EEDEC02F000D000D0D0
:100640000000E450E82EF6D7120000C0E5FF01C01C
:10065000E5FF02C0E5FF0001A56B05010051E83888
:10066000E840030B006E005002E0E86A12D105EE8C
:1006700001F0EFCF00F0005001E103D10050010A7A
:1006800001E1FFD00050030A01E1FBD00050050A50
:1006900001E1CED00050060A1CE00050080A0DE02F
:1006A0000050090A01E1C7D000500A0A01E1E9D06F
:1006B00000500B0A01E1E5D0E1D0000E0001916F7E
:1006C0005E0E906F800E926F010E0001986F996B15
:1006D000D8D005EE03F0EFCF00F0010E005CD8A0FB
:1006E000A3D0040E005CD8B09FD0000603C0E5FF85
:1006F00004C0E5FF046A00340436E8340436FC0B19
:10070000036E000EFB6E070EFA6E220E03260450D7
:10071000FA22D8B0FB2A0350E4CF04F0E4CF03F070
:10072000F96E97EF03F0AEEF03F0E4EF03F078C05B
:1007300090F079C091F07AC092F078C000F079C062
:1007400001F07AC002F000C0E9FF01C0F3FF0250DF
:10075000F1EC0BF00001986F996B93D005EE02F06D
:10076000EFCF00F00050030DF3CF00F0F4CF01F015
:1007700000017B5100267C5101227D51026A022238
:1007800000C0E9FF01C0F3FF0250AFEC0BF0000125
:10079000906FF3CF91F0F4CF92F090C000F091C041
:1007A00001F092C002F0020E0026000E0122022289
:1007B00000C0E9FF01C0F3FF0250CAEC0BF00001DA
:1007C000986FF3CF99F05DD005EE02F0EFCF00F017
:1007D0000050030DF3CF00F0F4CF01F000017E5183
:1007E00000267F5101228051026A022200C0E9FFE7
:1007F00001C0F3FF0250AFEC0BF00001906FF3CF9C
:1008000091F0F4CF92F090C000F091C001F092C04E
:1008100002F000C0E9FF01C0F3FF0250F1EC0BF061
:100820000001986F996B2DD0010E0001A56F29D0A2
:10083000040E5F6E26D078C000F079C001F07AC057
:1008400002F0110E0026000E0122022200C0E9FF74
:1008500001C0F3FF0250F1EC0BF0006E05EE02F068
:10086000EFCF01F00150005C05E3EFCFA4F0060EDE
:100870005F6E07D0010E0001A56F03D0010E0001CD
:10088000A56F0001A551D880E866D890006A0036AF
:100890000050E4CF02F0E4CF01F0E4CF00F012000A
:1008A00000C0E5FF01C0E5FF02C0E5FF03C0E5FFB2
:1008B00004C0E5FF5F50040A0BE105EE02F0EFCF44
:1008C0006EFF6E5003E0050E5F6E02D0030E5F6E8A
:1008D0000001A351010A29E1000E016E900E006E85
:1008E000800E026E000E046E980E036E800EE56E92
:1008F0000450E56E0350E56EE56A080EE56E0250A1
:10090000E56E0150E56E0050E56E000EE56A7BEC89
:1009100007F0090EE126040104BD03D0C80E046FE0
:1009200006D0880E0401046F02D094EC0BF05F50E7
:10093000060A01E0CCD0716A726A736A746A756AD9
:10094000766A776A786A796A7A6A7B6A7C6A7D6A8B
:100950007E6A7F6A030E0001A45D1DE2AC0E0001F9
:10096000846F040E856F000E866F160E00018D6F6A
:10097000050E8E6F000E8F6F800E00018A6F050EC0
:100980008B6F000E8C6FBA0E0001876F050E886F9B
:10099000000E896F3CD00A0EF66E200EF76E000E28
:1009A000F86E0900F5CF84F00900F5CF85F0090055
:1009B000F5CF86F00D0EF66E200EF76E000EF86E77
:1009C0000900F5CF8DF00900F5CF8EF00900F5CFC5
:1009D0008FF0100EF66E200EF76E000EF86E090006
:1009E000F5CF8AF00900F5CF8BF00900F5CF8CF038
:1009F000130EF66E200EF76E000EF86E0900F5CF9E
:100A000087F00900F5CF88F00900F5CF89F0A4C080
:100A10005EF00001A45103E1050E5F6E58D00F0E89
:100A20000001A66F0001A65103E0010E006E01D087
:100A3000006A0050D8B449D00001A451030DF3CF8F
:100A400000F0F4CF01F0000184510026855101220D
:100A50008651026A022200C0E9FF01C0F3FF025082
:100A6000AFEC0BF0006EF3CF01F0F4CF02F0000119
:100A7000A651030DF3CF03F0F4CF04F0035000268A
:100A800004500122E86A022200C0E9FF01C0F3FF1E
:100A90000250AFEC0BF0006EF3CF01F0F4CF02F098
:100AA000F2CFE5FFF29E0500C40EFD6E0A0EFE6E4B
:100AB000000EFF6EE450F26E02C0FBFF01C0FAFFB1
:100AC0000050F96E0001A607ADD7070E5F6EE4CFA8
:100AD00004F0E4CF03F0E4CF02F0E4CF01F0E4CF80
:100AE00000F01200D9CFE5FFE1CFD9FF00C0E5FF4C
:100AF00001C0E5FF02C0E5FF03C0E5FF04C0E5FF5C
:100B000005C0E5FF06C0E5FF07C0E5FF020EDBCF2D
:100B100000F0030EDBCF01F0040EDBCF02F0050E78
:100B2000DBCF03F0060EDBCF04F0070EDBCF05F0C2
:100B3000080EDBCF06F0090EDBCF07F000500001F6
:100B4000646F0150656F0250666F0350676F045009
:100B50000001686F0550696F06506A6F07506B6F30
:100B60000001645100016A03F3CF00F0F4CF01F0FB
:100B7000005000016E6F01506F6F00016451000161
:100B80006803F3CF00F0F4CF01F0005000016C6F68
:100B900001506D6F0001675100016803F3CF00F051
:100BA00000016F51002600506F6F00016651000177
:100BB0006903F3CF00F000016F51002600506F6F02
:100BC0000001665100016803F3CF00F0F4CF01F09B
:100BD00000016E5100266F51012200506E6F0150CE
:100BE0006F6F0001655100016903F3CF00F0F4CF8E
:100BF00001F000016E5100266F51012200506E6F0E
:100C000001506F6F0001655100016A03F3CF00F0DE
:100C100000500001736F0001655100016803F3CFBC
:100C200000F0F4CF01F000500001716F0150726FBD
:100C30000001645100016B03F3CF00F0005000018C
:100C4000776F0001645100016903F3CF00F0F4CF26
:100C500001F000500001756F0150766F0001706B5C
:100C60000001746B0001705100016C25006E0001E1
:100C7000715100016D21016E0001725100016E2160
:100C8000026E0001735100016F21036E00506C6F02
:100C900001506D6F02506E6F03506F6F0001745101
:100CA00000016C25006E0001755100016D21016E7F
:100CB0000001765100016E21026E000177510001A2
:100CC0006F21036E03C0E9FF02C0F4FF01C0F3FF10
:100CD0000050E4CF07F0E4CF06F0E4CF05F0E4CF16
:100CE00004F0E4CF03F0E4CF02F0E4CF01F0E4CF6E
:100CF00000F0E4CFD9FF1200D9CFE5FFE1CFD9FF53
:100D000000C0E5FF01C0E5FF02C0E5FF03C0E5FF4D
:100D100004C0E5FF05C0E5FF06C0E5FF07C0E5FF2D
:100D200080B804D00A0EF9EC02F0FF0009C4A8F064
:100D3000010E0001A85DD8A0C2D010C500F0060EBB
:100D4000005CD8B0A7D008C0E5FF09C0E5FF096A7C
:100D500000340936E8340936FC0B086E000EFB6ED1
:100D60000D0EFA6E7C0E08260950FA22D8B0FB2A26
:100D70000850E4CF09F0E4CF08F0F96ECAEF06F0AE
:100D8000D3EF06F0E2EF06F036EF07F037EF07F0AB
:100D90003CEF07F011C5F6FF12C5F7FF13C5F8FFCA
:100DA000E0EC0BF080D011C5F6FF12C5F7FF13C5BC
:100DB000F8FF050EE56E140EE56E42EC0BF0020E28
:100DC000E12671D0400E00019A6F9B6B11C500F0B7
:100DD000016A12C502F0036A0350E56E0250E56E27
:100DE000010EE56E000EE56E55EC0AF0026EF3CFD3
:100DF00003F0040EE126025000260350012213C521
:100E000002F0036A046A056A0550E56E0450E56E57
:100E10000350E56E0250E56E000EE56E010EE56EC4
:100E2000000EE56E000EE56E72EC05F0026EF3CF7B
:100E300003F0F4CF04F0E9CF05F0080EE126E86AEC
:100E400001BEFF0E066E076E0050022601500322FF
:100E5000065004220750052204500001956F0350EC
:100E6000946F0250936FA5EC0AF01DD01CD00A0EAF
:100E7000F9EC02F0FF0017D0160E00019A6F9B6B81
:100E8000C40E0001936F050E946F000E956FA5ECD4
:100E90000AF009D0400E0401096F100E0A6F050E0A
:100EA0000B6F840E086F400E0401096F08BD03D05C
:100EB000C80E086F0DD0880E0401086F09D0400ECF
:100EC0000401096F100E0A6F050E0B6F840E086F78
:100ED000E4CF07F0E4CF06F0E4CF05F0E4CF04F070
:100EE000E4CF03F0E4CF02F0E4CF01F0E4CF00F070
:100EF000E4CFD9FF1200D9CFE5FFE1CFD9FF00C081
:100F0000E5FF01C0E5FF02C0E5FF03C0E5FF04C047
:100F1000E5FF05C0E5FF06C0E5FF07C0E5FF08C027
:100F2000E5FF09C0E5FF0AC0E5FF0BC0E5FF020EC3
:100F3000DBCF00F0030EDBCF01F0040EDBCF02F0BD
:100F4000050EDBCF03F0060EDBCF04F0070EDBCF80
:100F500005F0080EDBCF06F0090EDBCF07F00A0E16
:100F6000DBCF08F006C0E9FF07C0F3FF0850CAEC6A
:100F70000BF0096EF3CF0AF005500A5C02E1045051
:100F8000095C05E209C096F00AC097F004D004C0DD
:100F900096F005C097F000500024046E0428040D5C
:100FA000F3CF00F0000E0024046E056A040E052243
:100FB000042AD8B0052A000196510B6E04C0E9FF3F
:100FC00005C0EAFF0BC0EFFF000E0026040E046A06
:100FD0000422020E0026D8B0042A00C0E9FF04C093
:100FE000EAFFEECF00F0EFCF04F004500001826F73
:100FF0000050816F800E836F00019651095E9751FA
:101000000A5A09C0E5FF0AC0F4FF06C0E9FF07C09D
:10101000F3FF08502BEC0CF0000196519711D8B457
:1010200042D081C000F082C004F083C005F001C04E
:10103000E9FF02C0F3FF0350AFEC0BF0066EF3CFF5
:1010400007F0F4CF08F006C0E9FF07C0F3FF08502F
:10105000F1EC0BF0096E09C0E5FF00C0E9FF04C028
:10106000F3FF055041EC0CF00001812B01E3822BD2
:1010700002E30001832B062AD8B0072AD8B0082A39
:1010800006C0E5FF07C0F4FF08C0F6FF01C0E9FF96
:1010900002C0F3FF035011EC0CF0FF0E0001962785
:1010A00001E29707B9D7E4CF0BF0E4CF0AF0E4CF21
:1010B00009F0E4CF08F0E4CF07F0E4CF06F0E4CF86
:1010C00005F0E4CF04F0E4CF03F0E4CF02F0E4CF86
:1010D00001F0E4CF00F0E4CFD9FF120000C0E5FF3B
:1010E00001C0E5FF02C0E5FF03C0E5FF04C0E5FF66
:1010F0000001A36B0001986B996B25EC03F0006E67
:101100000050D8B46AD06D98006A050100BF002A6B
:101110000050010A01E04ED0010E0001A36F080E3D
:101120000401016F000E006E050E016E0050026F8B
:101130000150036F800E006F080E006E050E016EE9
:101140000050066F0150076F05EE06F0EECF00F07D
:10115000EFCF01F000019951015C02E19851005C70
:1011600006E205EE06F0EECF98F0EFCF99F0000E14
:10117000016E900E006E800E026E000E046E980ED0
:10118000036E800EE56E0450E56E0350E56EE56A71
:10119000080EE56E0250E56E0150E56E0050E56EFA
:1011A000000EE56A7BEC07F0090EE126C80E04018B
:1011B000046F22D0020E0001A36F080E0401016F1C
:1011C000080E006E050E016E0050026F0150036F95
:1011D000C80E006F056B046F0FD06D98080E0401E8
:1011E000016F000E006E050E016E0050026F01507F
:1011F000036F840E006F046FE4CF04F0E4CF03F0BC
:10120000E4CF02F0E4CF01F0E4CF00F0120000C020
:10121000E5FF0001606B616B080E626F636B00019C
:10122000605161116211631106E0FF0E60276123B6
:1012300062236323F4D7000EF66E200EF76E000EC5
:10124000F86E0900F5CF00F000502EE1010EF66EA9
:10125000200EF76E000EF86E0900F5CF78F0090049
:10126000F5CF79F00900F5CF7AF0040EF66E200E76
:10127000F76E000EF86E0900F5CF7BF00900F5CF90
:101280007CF00900F5CF7DF0070EF66E200EF76EAC
:10129000000EF86E0900F5CF7EF00900F5CF7FF063
:1012A0000900F5CF80F015D0840E0001786F030E91
:1012B000796F000E7A6FC80E00017B6F030E7C6F92
:1012C000000E7D6F3A0E00017E6F040E7F6F000EE0
:1012D000806FAC0E0001846F040E856F000E866F68
:1012E000160E00018D6F050E8E6F000E8F6F800E33
:1012F00000018A6F050E8B6F000E8C6FBA0E000115
:10130000876F050E886F000E896FE4CF00F0120022
:1013100000C0E5FF01C0E5FF02C0E5FF03C0E5FF37
:1013200004C0E5FF686A7B0E696E6B6A6E6A68A628
:1013300002D06896FCD7030E5F6E5E6A5D6A706AC3
:10134000716A726A736A746A756A766A776A786AA9
:10135000796A7A6A7B6A7C6A7D6A7E6A7F6A6D983E
:10136000100E0001A26F84C000F085C001F086C09D
:1013700002F000C0E9FF01C0F3FF0250AFEC0BF038
:10138000006EF3CF01F0F4CF02F00001A205030DCF
:10139000F3CF03F0F4CF04F00350002604500122F1
:1013A000E86A022200C0E9FF01C0F3FF0250AFEC7F
:1013B0000BF0006EF3CF01F0F4CF02F0F2CFE5FFB7
:1013C000F29E0500E00EFD6E130EFE6E000EFF6E27
:1013D000E450F26E02C0FBFF01C0FAFF0050F96E4C
:1013E0000001A207A251D8A4BED7100EA26FE4CF6D
:1013F00004F0E4CF03F0E4CF02F0E4CF01F0E4CF57
:1014000000F0120000C0E5FF01C0E5FF02C0E5FFEB
:1014100003C0E5FF04C0E5FF00019A519B1104E100
:101420000001A851D8A436D0000E00019B5D02E156
:10143000400E9A5DD8700001A86BA83700019A5140
:101440000401156F000E016E930E006E800E026E89
:10145000000E046E9A0E036E800EE56E0450E56E6B
:101460000350E56EE56A400EE56E0250E56E0150F0
:10147000E56E0050E56E020EE56E7BEC07F0090E9E
:10148000E126040114BD03D0C80E146F03D0880EEA
:101490000401146FE4CF04F0E4CF03F0E4CF02F0D2
:1014A000E4CF01F0E4CF00F01200D9CFE5FFE1CFA7
:1014B000D9FF00C0E5FF01C0E5FF02C0E5FF03C0A2
:1014C000E5FF020EDBCF00F0030EDBCF01F0040ED0
:1014D000DBCF02F0050EDBCF03F0005000019C6F64
:1014E00001509D6F025000019E6F03509F6F0001DD
:1014F0009C5100019E03F3CF00F0F4CF01F00050A7
:101500000001A06F0150A16F00019C5100019F03D9
:10151000F3CF00F000019D5100019E03F3CF01F0D5
:10152000015000260001A15100260050A16FA1C06A
:10153000F3FFA051E4CF03F0E4CF02F0E4CF01F0D9
:10154000E4CF00F0E4CFD9FF120000C0E5FF01C0F6
:10155000E5FF02C0E5FF03C0E5FF04C0E5FF000EA4
:1015600000019B5D02E1400E9A5DD8700001A86BFE
:10157000A83700019A510401156F500E166F050E21
:10158000176F000E016E930E006E800E026E000E3D
:10159000046E9A0E036E800EE56E0450E56E0350E5
:1015A000E56EE56A400EE56E0250E56E0150E56EAF
:1015B0000050E56E020EE56E7BEC07F0090EE126A9
:1015C000040114BD03D0C80E146F03D0880E0401AB
:1015D000146FE4CF04F0E4CF03F0E4CF02F0E4CFE3
:1015E00001F0E4CF00F012009298808807EC09F037
:1015F00002EC0CF0C00E006E270E016E090E026E9A
:10160000036A51EC0CF03DEC00F0000EF66E200E7B
:10161000F76E000EF86E0900F5CF04F0045003E0F9
:101620000450010AEEE1FF0E0026012202220322ED
:101630000050011002100310E4E192988098160EF9
:10164000F66E200EF76E000EF86E0900F5CF00F072
:101650000900F5CF01F00900F5CF02F0F2CFE5FF68
:10166000F29E0500800EFD6E160EFE6E000EFF6EE1
:10167000E450F26E02C0FBFF01C0FAFF0050F96EA9
:10168000FFD71200D9CFE5FFE1CFD9FF00C0E5FFBA
:1016900001C0E5FF020EDBCF00F0030EDBCF01F04F
:1016A0000A000001A96B200E0001A95D0DE200C037
:1016B000E9FF01C0EAFFEFCFF5FF002AD8B0012A09
:1016C0000F000001A92BEFD7A68EA69CA684F29E40
:1016D000550EA76EAA0EA76EA682E4CF01F0E4CF46
:1016E00000F0E4CFD9FF1200E8AE0AD0F3CFEAFF52
:1016F000EE50EECFF3FFEECFF4FFEECFE9FF120096
:10170000E8BC11D0E9CFF6FFF3CFF7FFF86E090080
:10171000F5500900F5CFF3FF0900F5CFF4FF0900FC
:10172000F5CFE9FF1200120000C0E5FF01C0E5FFA0
:101730000001A36B080E0401016F000E006E050E80
:10174000016E0050026F0150036F880E006F046B32
:10175000160E706EE4CF01F0E4CF00F01200E8AE98
:1017600008D0F3CFEAFFEE50EECFF3FFEECFF4FF59
:101770001200E8BC0ED0E9CFF6FFF3CFF7FFF86E0A
:101780000900F5500900F5CFF3FF0900F5CFF4FF8C
:1017900012001200E8AE06D0F3CFEAFFEE50EECF13
:1017A000F3FF1200E8BC0BD0E9CFF6FFF3CFF7FF51
:1017B000F86E0900F5500900F5CFF3FF1200120092
:1017C000D9CFE5FFE1CFD9FFA68EA69CA684A68837
:1017D000F29E550EA76EAA0EA76EA682E4CFD9FF81
:1017E0001200E8AE04D0F3CFEAFFEE501200E8BCDE
:1017F00008D0E9CFF6FFF3CFF7FFF86E0900F550F8
:1018000012001200696A140E6F6E080E6D6E6DBACA
:10181000FED7686A110E696E020E5F6E5E6A5D6ABF
:101820001200E8AE09D0F3CFEAFFE4CFEEFFF4CF29
:10183000EEFFF6CFEEFF1200E8AC12001200400EF1
:101840000401096F100E0A6F050E0B6F880E086FEA
:101850001C0E716E1200E8AE07D0F3CFEAFFE4CFA2
:10186000EEFFF4CFEEFF1200E8AC1200120012EE11
:10187000FEF022EEFEF0F86AA68EA69CF4EC0AF0CA
:10188000FFD7E8AE05D0F3CFEAFFE4CFEEFF1200BA
:10189000E8AC12001200480E0401146F1A0E726EAA
:0E18A00012006DA202D0A08AA19A12001200BE
:10200000FF000000000000000000000000000000D1
:0A20100000000000000000000000C6
:10202000E8CFE5FFD8CFE5FFE0CFE5FFF3CFE5FF51
:10203000F4CFE5FFE9CFE5FFEACFE5FFFACFE5FF13
:10204000FBCFE5FFE4CFFBFFE4CFFAFFE4CFEAFFED
:10205000E4CFE9FFE4CFF4FFE4CFF3FFE4CFE0FF08
:0A206000E4CFD8FFE4CFE8FF100042
:10400000E8CFE5FFD8CFE5FFE0CFE5FFF3CFE5FF51
:10401000F4CFE5FFE9CFE5FFEACFE5FFFACFE5FF13
:10402000FBCFE5FFE4CFFBFFE4CFFAFFE4CFEAFFED
:10403000E4CFE9FFE4CFF4FFE4CFF3FFE4CFE0FF08
:0A404000E4CFD8FFE4CFE8FF100042
:020000040030CA
:0E000000240E3F1EFF8181FF0FC00FA00F4096
:00000001FF
